:020000040008F2
:0400000018F09FE570
:04002000880008004C
:100040000120704770B50E4E0E4C82B03500361D43
:1000500005E00100306800F005F90C350C36A542CA
:1000600009D2706831682A688842F2D1306800216C
:1000700000F006F9F1E702B070BC01BC0047C046D1
:10008000A4020800B002080000000FE11F00C0E356
:10009000120080E300F021E114D09FE51F00C0E3CF
:1000A0001F0080E300F021E108D09FE508009FE5F4
:1000B00010FF2FE14002010000020100C000080013
:1000C00001C08FE21CFF2FE1044C054D054E064F89
:1000D000AE462047002809D0BE4630474100080000
:1000E000D500080045000800ED000800044C054D4F
:1000F0000020AE462047044C044DAE462047000089
:10010000E1010800F7000800550208009902080004
:1001100000B5401E0028FCD101BC004700B52149B4
:1001200020220A60002801D4401EFBE701BC0047E2
:1001300000B50948FFF7F2FF0848802189000160F7
:100140000748132101600748132101600648012177
:10015000016001BC0047C046204E00003405FFFF8F
:100160000006FFFF0806FFFF8C04FFFF10B5040028
:1001700009482406240E04600A48A32101600748A8
:1001800000680028FBD0FA208000FFF7C1FF044878
:10019000006810BC02BC08470405FFFF0C05FFFF08
:1001A0001005FFFF0005FFFF00B5002801D1084A38
:1001B0001160012801D1074A1160022801D1064AC5
:1001C0001160032801D1054A116001BC0047C046F7
:1001D0000406FFFF0C06FFFF1406FFFF1C06FFFFCF
:1001E00000B500F013F8FFF7A3FF00F01FF80020A0
:1001F000FFF7BCFF01000020FFF7D6FF0120FFF74B
:10020000B5FF01000120FFF7CFFFF0E7044801210F
:1002100001600448022101600348F4210160704735
:100220000404FFFF0804FFFF0C04FFFF0248C02185
:10023000890401607047C04660F4FFFF704700000A
:1002400010B582B00400009469460120FFF7F6FF64
:10025000F9E7000000B581B000F01EF801B001BC64
:100260000047000010B40300002A05D00C78491C98
:100270001C705B1C521EF9D110BC00B0704700000E
:100280000906090E0300002A03D019705B1C521ED8
:10029000FBD100B070470000014CA646204700008B
:1002A0004102080000000000000001000000010001
:0400000500080000EF
:00000001FF
